:020000040000FA
:10000000B00A0020150200003F020000410200007B
:10001000430200004502000047020000000000000B
:100020000000000000000000000000004902000085
:100030004B020000000000004D0200004F020000D3
:100040005102000051020000390500005102000079
:1000500051020000000000005102000051020000A7
:100060005102000051020000510200005102000044
:100070005102000051020000510200005102000034
:100080005102000051020000510200005102000024
:100090005102000051020000510200005102000014
:1000A00051020000510200000000000000000000AA
:1000B000510200005102000000000000000000009A
:1000C0000000000000000000000000000000000030
:1000D0000000000000000000000000000000000020
:1000E0000000000000000000000000000000000010
:1000F0000000000000000000000000000000000000
:1001000000000000000000000000000000000000EF
:1001100000000000000000000000000000000000DF
:1001200000000000000000000000000000000000CF
:1001300000000000000000000000000000000000BF
:1001400000000000000000000000000000000000AF
:10015000000000000000000000000000000000009F
:10016000000000000000000000000000000000008F
:10017000000000000000000000000000000000007F
:10018000000000000000000000000000000000006F
:10019000000000000000000000000000000000005F
:1001A000000000000000000000000000000000004F
:1001B000000000000000000000000000000000003F
:1001C000000000000000000000000000000000002F
:1001D000000000000000000000000000000000001F
:1001E000000000000000000000000000000000000F
:1001F00000000000000000000000000000000000FF
:10020000DFF80CD000F042F800480047ED0900008C
:10021000B00A00200F4800680F4909680A280AD16F
:10022000002908D10D4802686FF070031A404FF0A2
:1002300040031A4302600A4880470A480047FEE725
:10024000FEE7FEE7FEE7FEE7FEE7FEE7FEE7FEE786
:10025000FEE700003001001034010010E40E004001
:10026000B10200000102000040EA01039B0703D035
:1002700009E008C9121F08C0042AFAD203E011F8E5
:10028000013B00F8013B521EF9D27047064C074D66
:1002900006E0E06840F0010394E807009847103456
:1002A000AC42F6D3FFF7B0FFF016000010170000C5
:1002B0002DE9F041914E4FF080548F4DD4F830210C
:1002C00030782B68511CC0F3031000D1DAB200273C
:1002D0004FF00108062A05D1B4F82413884AC1F367
:1002E00004211160D9B2062904D1032802D186491C
:1002F0008448486700F0E6FB28B1D4F844028349FB
:10030000C0F342300860297830780629C0F3031022
:1003100006D1032804D17E48016821F08071016074
:1003200000F0EEFB40B14FF08040C0F80C71C0F817
:1003300010717648001F076029683078CAB2C0F390
:100340000310062A05D1032803D1704B032264331E
:100350001A60C9B206290ED103280CD16D4A0521B5
:1003600011606C497831C1F800806A480830076034
:10037000111D3F20086000F0E1FBE8B3664800680B
:10038000664908606448001D0068091D08606248ED
:1003900008300068091D08605F480C300068091DBE
:1003A00008605D4810300068091D08605A48143024
:1003B0000068091D08605848183000685749203106
:1003C000086055481C300068091D086052482030FC
:1003D0000068091D0860504824300068091D086045
:1003E0004D4828300068091D08604B482C300068D3
:1003F000091D0860484800E018E0303000684749AF
:1004000040310860444834300068091D08604248A3
:1004100038300068091D08603F483C300068091DFD
:1004200008603D4840300068091D0860D4F830017C
:10043000411C00D128783A4D062804D1D4F858023E
:1004400000F04F00286000F01FFB30B13548016814
:10045000C90702D06FF001010160D4E94C100629F0
:1004600007D1C21E022A04D92F4A136843F48063BD
:1004700013600A2905D1020003D02A6842F00F0256
:100480002A604FF01022062907D1C01E032804D984
:10049000D2F808021D491C310860D2F80002234B33
:1004A000002803DBD2F8040200280EDA012000F055
:1004B000CFFE1520C2F8000219680029FCD0C2F84E
:1004C000040218680028FCD00BE092F80C02C00768
:1004D0000CD0012000F0BCFEC2F80C721868002895
:1004E000FCD0002000F0B4FE00F034F811491048B0
:1004F0000860BDE8F0810000E00F00F0E80F00F0B8
:10050000403501400DF0ADBA00C007403C05004049
:10051000FCED00E0105600400404001020C500402F
:10052000E40E0040000400403C17004000E401409D
:100530000090D00338000020014800680047000008
:100540000C000020014A024900F025B855090000BE
:1005500034000020BFF34F8F05480168054A01F4BD
:10056000E06111430160BFF34F8F00BFFDE7000062
:100570000CED00E00400FA0502E008C8121F08C1F3
:10058000002AFAD170477047002001E001C1121F14
:10059000002AFBD170472DE9F04116460F4604466C
:1005A000002503E03946B047641C6D1C2078002804
:1005B000F8D12846BDE8F08172B609480068C00746
:1005C00000D000BEBFF34F8F0548E4380168054AEC
:1005D00001F4E06111430160BFF34F8F00BFFDE7FD
:1005E000F0ED00E00400FA050EB500210091CDE920
:1005F00001106A4644F20100FFF7DEFF0EBD10B5A0
:100600008268C368934203D000F091F9002010BDC6
:10061000052010BD29B112B1531E134203D0092089
:1006200070470E2070470160838000218160C160A7
:100630000846704710B58268C3689A1A83889A4240
:1006400003D800F07EF9002010BD042010BD00008A
:1006500070B50A4E01460A48B578FFF7D0FF044648
:100660004DB10020B070711C0122C81D00F0BCFA11
:1006700008B1FFF7B9FF204670BD0000140000204C
:100680008C020020F0B5244E89B01F460D000446B0
:1006900072603FD0A888296882B22048FFF7BAFF6D
:1006A000002835D1A889A96882B21C481030FFF70C
:1006B000B1FF00282CD1202219496846FFF7D4FD4C
:1006C00060690690207C00B101208DF814008DF83F
:1006D0001C70607C00B10E208DF81500E06802905F
:1006E000A068039020680190606800900A480D4A55
:1006F0006946083000F044FA002809D1B07020683B
:10070000401C05D004490122491CC81D00F06CFAA8
:1007100009B0F0BD0720FBE7140000208C02002088
:10072000D01600006513000010B501461048FFF711
:1007300081FF040019D10F480F4A0178515C19B1AB
:10074000001D00F077FD02E00C3000F04DFC60B9B8
:10075000084907480839FFF752FF30B90549012217
:100760000839044800F050FA0446204610BD000045
:100770009C0200201C0000200000002000F002B8B5
:1007800000F008B872B602480168491C0160704761
:100790003000002003490868401E086000D162B69E
:1007A00070470000300000202DE9F041064608683F
:1007B0000C46411C4FF0A0474FF0010506D005FA4A
:1007C00000F1C7F80815206800F076FA6068411C4F
:1007D00002D0002100F05EFA3168A069C1F824055A
:1007E000607D227D31681043C1F86C05D4E90012A8
:1007F0003068C0F81425C0F80C15207D012815D1EB
:10080000A068411C02D0002100F044FAE068411CBD
:1008100005D08540C7F80855E06800F04DFAD4E9E6
:1008200002123068C0F80825C0F81015BDE8F08144
:100830002DE9F041064608680C46411C4FF0A047E0
:100840004FF0010506D005FA00F1C7F80815206839
:1008500000F03CFA6068411C02D0002100F023FA4D
:100860003168A069C1F82405607D217D32680843A4
:10087000C2F86C05D4E900123068C0F80C15C0F855
:100880001425207D012815D1A068411C02D000212B
:1008900000F009FAE068411C05D08540C7F808550A
:1008A000E06800F013FAD4E902123068C0F80825B5
:1008B000C0F81015BDE8F0812DE9FC410646C007DF
:1008C0004FF000050ED0104F00240122385D009536
:1008D00000231146019500F0A7F9641C042CF4D301
:1008E00000F01CF8B0070DD5074E0024361D00227D
:1008F000305D032300951146019500F095F9641CC5
:10090000042CF4D3BDE8FC81C01600000249085C49
:10091000012100F0E5B90000C016000010B5002468
:100920002046FFF7F3FF641C042CF9D310BD826846
:1009300083881A4003689A5C0A708168491C816048
:100940007047C26883881A4003689954C168491C7B
:10095000C160704710B50446C0B2FFF7E5FE2046FF
:1009600010BD000070B50D46044600684FF4887154
:1009700000F0D7F94FF49071206800F0D2F94FF4ED
:100980009271206800F0CDF94FF4A271206800F058
:10099000C8F94FF4AC71206800F0C3F9206812491F
:1009A000C0F804132068690740F30730090E0028D7
:1009B00004DB00F1E02080F8001405E000F00F00F7
:1009C00000F1E02080F8141D206840F30730002873
:1009D00009DB00F01F02012191404009800000F175
:1009E000E020C0F8001170BD100342008AB0012061
:1009F000FFF762FF182216496846FFF735FC1548D5
:100A0000069015494FF48070CDE90701099007233E
:100A1000124A06A96846FFF735FE08B1FFF7E4FD64
:100A20000FA0FFF78FFD06A8FFF712FE0028FAD1EE
:100A30009DF81800FFF778FE0028F9D19DF81800FE
:100A4000712801D05128EED10CA0FFF77BFDFEE705
:100A5000A81600003C0000203C01002053130000B9
:100A60000D0A55415254206578616D706C65207394
:100A70007461727465642E0D0A000000200D0A4531
:100A8000786974210D0A00004FF08050D0F83011C1
:100A90004A1C07D0D0F8340106290ED00A2909D003
:100AA0000020704706480178054808300078C0F3F8
:100AB0000310F1E708B10128F3D0012070470000CE
:100AC000E00F00F04FF08050D0F830114A1C07D0F2
:100AD000D0F8340106290ED00A2909D00020704729
:100AE00006480178054808300078C0F30310F1E7A4
:100AF00008B10128F3D0012070470000E00F00F09A
:100B00004FF08050D0F830114A1C07D0D0F8340193
:100B100006290ED00A2909D000207047064801781E
:100B2000054808300078C0F30310F1E708B1012848
:100B3000F3D0012070470000E00F00F04FF080502C
:100B4000D0F830114A1C06D0D0F8340106290AD05A
:100B50000A290CD010E009480178084808300078CC
:100B6000C0F30310F2E7C01E012803D804E008B167
:100B7000012800D00120704700207047E00F00F0EE
:100B8000F0B505460478154889B0164640F824208B
:100B9000124A0869121DA2F1080742F82400487F92
:100BA000385520226846FFF75FFB04942878385CAC
:100BB00048B10EB10A4A00E000226946281D00F043
:100BC0002BFA09B0F0BD0EB1064A00E000226946DA
:100BD00005F10C0000F0D4F8F3E700000400002059
:100BE000651500000914000030B40378054CE35C7F
:100BF0001BB130BC001D00F045BA30BC0C3000F019
:100C000029B900000000002030B40378054CE35CF3
:100C10001BB130BC001D00F0B7BA30BC0C3000F086
:100C20008FB900000000002070B541EA4201DDE903
:100C300004564FF0A04441EA830141EA052104EB48
:100C4000800041EA0641C0F8001770BD70B541EA66
:100C50004201DDE904564FF0A04441EA830141EA34
:100C6000052104EB800041EA0641C0F8001770BD81
:100C700070B541EA4201DDE904564FF0A04441EA73
:100C8000830141EA052104EB800041EA0641C0F8F6
:100C9000001770BD1CB500220B4600921146019250
:100CA000FFF7D4FF1CBD1CB500220B460092114675
:100CB0000192FFF7DDFF1CBD1CB5002100910B4622
:100CC000012201911146FFF7C1FF1CBD1CB5002197
:100CD00000910B46012201911146FFF7C9FF1CBD8F
:100CE00001224FF0A043824011B1C3F8082570479C
:100CF000C3F80C2570474058002800D001207047E9
:100D000008B5002242504058009008BDD0F80403B6
:100D1000084000D0012070474058002800D0012032
:100D2000704708B5002242504058009008BD01218C
:100D3000B1EB507F01D1012070470020704770B5A2
:100D40000D4600F091FA04000FD00020FFF716FDC9
:100D5000207920B10020FFF713FD112070BD012084
:100D6000256020710020FFF70BFD002070BD000002
:100D70000149024800F060BB3C0200200020004016
:100D80002DE9F0410546007916460F4600EB40017B
:100D90002D4A01EBC00102EB810494F82A1011B135
:100DA0000820BDE8F081294951F820102868FFF794
:100DB000C6FF08B11120F4E739462846FFF7F4FCD6
:100DC00066603869206030004FF001062FD03F7F09
:100DD0004FF48E712868FFF793FF4FF4A2712868D3
:100DE000FFF78EFF28681A49C0F8041328684FEAF5
:100DF000471140F30730002804DB00F1E02080F8C1
:100E0000001405E000F00F0000F1E02080F8141D50
:100E1000286840F30730002809DB00F01F0106FABC
:100E200001F14009800000F1E020C0F800112868BD
:100E30000421C0F800150020A061E06184F82900B9
:100E400044F8140FA675ACE73C020020C816000059
:100E5000800002002DE9F05F054600794FF401762D
:100E600000EB400303EBC000344B03EB8004002095
:100E7000636813B12B68C3F80863A3694FF00009D6
:100E80006BB1E06938B1606810B12868C0F80463DC
:100E90001120BDE8F09FE2610120216105E0C4F866
:100EA0002490A261E160C4F81C9094F829100143D9
:100EB00002D1284600F013FA60680028286803D0A1
:100EC000C0F804630020E4E74FF4A2763146FFF750
:100ED00017FFB2464FF4927B59462868FFF70BFF85
:100EE00006464FF484712868FFF705FF8046514697
:100EF0002868FFF700FF074648EA07003043EBD0B9
:100F000056EA070007D12146286800F0B9F9A1691F
:100F1000606A8142E0D8C4F818900EB10320B8E7A7
:100F20000FB10F20B5E794F8291001200029296896
:100F300001D00860C6E74860C4E700003C0200201A
:100F40002DE9F05F054600790B4600EB400101EB0F
:100F5000C000244901EB8004284600F045F810B198
:100F60001120BDE8F09F62614FF00009C4F82090A5
:100F7000A36084F828904FF48E784E464146286846
:100F8000FFF7BEFE28684FF0010AC0F808A021460E
:100F9000286800F0B4F9606808BBD5F800B067694C
:100FA0000FE000BF94F8280008B10F2615E0414675
:100FB0005846FFF7A0FE0028F4D02146584600F01E
:100FC0009EF9206AB842F2D3574641462868FFF797
:100FD00092FE0028F9D02868C760C4F81490304603
:100FE000BFE700003C020020007900EB400101EB6C
:100FF000C000044901EB80004069002800D00120B6
:10100000704700003C0200200149024800F0C2BACB
:1010100068020020002000402DE9F04105461646F8
:1010200000790F46154A00EBC00102EB810494F8E9
:10103000201011B10820BDE8F081114951F82010AD
:101040002868FFF77CFE08B11120F4E739462846EE
:10105000FFF7EEFB6660386920601EB1397F2846D5
:10106000FFF780FC28680821C0F800150020A06167
:10107000E0616061012184F82010DCE76802002053
:10108000CC1600002DE9F05F044600790E4600EB17
:10109000C001DFF8F0A017460AEB81053046FFF7E4
:1010A00046FEB0B168684FF000084FF4047910B103
:1010B0002168C1F80893A8694FF0000B80B1E86976
:1010C00048B1686810B12068C0F804931120BDE8E9
:1010D000F09F1020FBE7EF614FF001082E6102E066
:1010E000EE60C5E9067B00254FF488712068FFF7A4
:1010F00018FE4FF4A2712068FFF713FE2068C0F8B5
:101100003465C0F838752068B8F1000F12D0D0F8F7
:10111000001241F02001C0F800122079D04600EB07
:10112000C0010AEB8100406838B12068C0F8049320
:101130002846CCE701210160EFE74FF4887A4FF4AD
:10114000A27951462068FFF7E7FD07464946206827
:10115000FFF7E2FD06464FF492712068FFF7DCFDD1
:10116000014647EA06000843EBD0227902EBC203AE
:1011700008EB8302C2F818B001B10325002ED7D0C6
:101180000F25D5E7680200202DE9F04704460E46FA
:101190000079274900EBC00001EB80051746304677
:1011A000FFF7C5FD30B1204600F044F820B1112012
:1011B000BDE8F0871020FBE76F61AE604FF49077D9
:1011C0004FF0000839462068FFF7ABFD4FF4AC76CE
:1011D00031462068FFF7A5FD2068AA686969C0F854
:1011E0004425C0F8481520684FF00109C0F8089060
:1011F0006868D0B9BA4651462068FFF78DFD0746AA
:1012000031462068FFF788FD0743F4D010B14FF056
:101210000F0808E02068C0F80C9031462068FFF7FE
:101220007BFD0028F9D0002068614046C0E700003F
:10123000680200200079054900EBC00001EB800046
:101240004069002800D0012070470000680200209B
:1012500003490860034801680029FCD0704700007A
:1012600004E5014000E401400349884201D10348FC
:101270007047002070470000002000400C00002054
:1012800070B5054688690C4600284FF484712846DD
:101290000AD0FFF735FDD5F81805626AE168885471
:1012A000606A401C606270BDFFF72AFDD5F8180522
:1012B00070BD1FB501238DF80030CDE90121D0E9C3
:1012C0000012684690471FBD1FB501238DF80030FE
:1012D000CDE90121D0E90012684690471FBD10B545
:1012E000044600684FF49271FFF70AFD4FF48471D1
:1012F0002068FFF705FD20680121016010BD70B571
:101300000C4605464FF48E71FFF7FAFC216AA0687F
:10131000415C206A401C2062C5F81C1570BD1FB5D9
:1013200000228DF800200291816801914261D0E98C
:101330000012684690471FBD1FB500228DF800209F
:101340000291816801914261D0E90012684690479C
:101350001FBD0178022901D0012902D14068FFF7A1
:1013600043B970477CB50178254DA1B301290BD055
:1013700002291DD18DF80010C068691C019001225E
:10138000C81DFFF731FC30E0017A59B1406801789F
:101390001C48FFF74FF91B4C012650B18DF8006037
:1013A00001900DE016490122491CC81DFFF71CFCE5
:1013B0007CBDA068E168814205D000208DF8000066
:1013C000696868468847A068E168081AA188884269
:1013D000E8D9AE707CBDFFE70A4809491030FFF735
:1013E0000EF930B103208DF800006968684688471F
:1013F000F0E70349012201F10800FFF705FCE9E7E6
:10140000140000208C0200201FB50A4601788DF8D8
:10141000001041680191017A8DF80810C0680390AE
:10142000044850F82210001F50F8222068469047C8
:101430001FBD0000080000202DE9FF470C460546AF
:101440004FF40071FFF762FC01274FF4017800268A
:1014500018B34FF4927949462846FFF74CFCE0B1A7
:1014600049462846FFF74CFCC5F8088394F8290044
:1014700000B96F6002208DF80000D5F88004C5F82F
:1014800080040390A0690290E0680190A661E66183
:10149000D4E900126846904728E004212846FFF767
:1014A00035FC18B34FF484712846FFF724FCE8B1EB
:1014B00021462846FFF7E4FE616AA069884215D1FB
:1014C000E06938B1E268616AA0612069E66166623C
:1014D000E06008E094F8290000B96F60C5F808835F
:1014E000A661E268616A2046FFF7E3FE4FF48E785A
:1014F00041462846FFF7FFFB80B16069216A8142BF
:1015000002D294F8280028B341462846FFF7F8FB9A
:10151000606918B161692046FFF701FF4FF4A278B6
:1015200041462846FFF7E7FB002818D041462846E9
:10153000FFF7E6FB94F8290000B12F60A0690028AE
:101540000DD0A661E268616A04B02046BDE8F047AC
:10155000FFF7AFBE21462846FFF7D1FEDEE7BDE824
:10156000FF8700001FB50A4601788DF8001041681A
:101570000191017A8DF80810C0680390044850F872
:101580002210001F50F82220684690471FBD00001F
:10159000080000202DE9FF410C464FF492770546E4
:1015A0003946FFF7B9FB0026B8B139462846FFF7A0
:1015B000B8FB02208DF80000D5F88004C5F880043F
:1015C0000390D5F83C050290E0680190A661E661C1
:1015D000D4E900126846904723E04FF488773946F3
:1015E0002846FFF799FBE0B139462846FFF799FBFB
:1015F000D5F83C15A069884213D1E06960B1E26872
:10160000D5F8000220F02000C5F80002E069A061D2
:101610002069E661E06001E0A661E2682046FFF72C
:1016200053FE4FF4A27739462846FFF775FB68B1A1
:1016300039462846FFF775FBA06938B1A661E66117
:10164000D5F83C152046E268FFF73EFE4FF4907651
:1016500031462846FFF760FB60B131462846FFF768
:1016600060FB0120E860606920B1D5F84C15204688
:10167000FFF762FE4FF4AC7631462846FFF74CFB8D
:1016800000280ED031462846FFF74BFB6069002842
:1016900007D0D5F84C1504B02046BDE8F041FFF75F
:1016A0004BBEBDE8FF8100000800000006000000FE
:1016B00005000000070000000000000000E0D70166
:1016C000111213140D0E0F10710D000009100000FF
:1016D000FFFFFFFFFFFFFFFFFFFFFFFFFFFFFFFF1A
:1016E00000000000000000000000D601060100001C
:1016F00010170000000000203C00000078050000EA
:101700004C1700003C000020740A0000880500000F
:1017100000000000000000000000000000000000C9
:1017200000000000000000000000000000000000B9
:1017300000200040000000000020004000000000E9
:0C17400000000000000000000090D0033A
:0400000500000201F4
:00000001FF
